:10007000436865636B73756D204661696C65640ADE
:1000800000436865636B73756D20537563636565C5
:050090006465640A0034
:100003008B098A0A890BE4FFD3ED9400EC9400403A
:100013001DAB09AA0AA90B1200A12FFFED1D700148
:0F0023001C7401250BF50BE4350AF50A80DA226F
:10003200E4F508F590759850438920758DDDD28ED0
:10004200D2997BFFFAF9FD7C401200038F088508E4
:1000520090E5086480600B7BFF7A0079701200BA29
:0E00620080CE7BFF7A0079811200BA80C32223
:0300000002009566
:0C009500787FE4F6D8FD75810B02003284
:1000A100BB010689828A83E0225002E722BBFE025D
:0900B100E32289828A83E4932290
:1000BA008B098A0A890BAB09AA0AA90B1200A1604B
:1000CA0013050BE50B7002050A14F91200A1FF12C1
:0E00DA0000E880E27F0A1200E87E007F00222C
:1000E800EFB40A07740D1200F3740A309811A89936
:1000F800B8130CC2983098FDA899C298B811F63078
:0701080099FDC299F599224F
:00000001FF
